:020000040800F2
:1000000000070020E504000881140008851400089A
:10001000DD14000885140008B1140008E704000886
:10002000E7040008E7040008E70400089D3500081D
:10003000E7040008E7040008E7040008E7040008F4
:10004000E7040008E7040008E7040008E7040008E4
:10005000E7040008E7040008AD390008D9390008B2
:10006000053A0008313A00085D3A0008E704000844
:10007000E7040008E7040008E7040008E7040008B4
:10008000E7040008E7040008E7040008B5230008B7
:100090002124000875240008C9240008893A0008B2
:1000A000E7040008E7040008E7040008E704000884
:1000B00019380008E7040008E7040008E70400080E
:1000C000E7040008E7040008E7040008E704000864
:1000D000E7040008E7040008E7040008E704000854
:1000E000F13A0008E7040008E7040008E704000804
:1000F000E7040008E7040008E7040008E704000834
:10010000E7040008E7040008E7040008E704000823
:10011000E7040008E7040008E7040008E704000813
:10012000E7040008E7040008E7040008E704000803
:10013000E7040008E7040008E7040008E7040008F3
:10014000E7040008E7040008E7040008E7040008E3
:10015000E7040008E7040008E70400086127000836
:10016000E7040008E7040008E7040008E7040008C3
:10017000E7040008E7040008E7040008E7040008B3
:10018000E7040008E7040008E7040008E7040008A3
:10019000E7040008E7040008E7040008E704000893
:1001A000E7040008E7040008E7040008E704000883
:1001B000E7040008E7040008E7040008E704000873
:1001C000E7040008E7040008E7040008E704000863
:1001D000E7040008E7040008E7040008E704000853
:1001E00053B94AB9002908BF00281CBF4FF0FF319E
:1001F0004FF0FF3000F074B9ADF1080C6DE904CE9A
:1002000000F006F8DDF804E0DDE9022304B07047F1
:100210002DE9F047089D04468E46002B4DD18A42B9
:10022000944669D9B2FA82F252B101FA02F3C2F1EC
:10023000200120FA01F10CFA02FC41EA030E94407D
:100240004FEA1C48210CBEFBF8F61FFA8CF708FB9E
:1002500016E341EA034306FB07F199420AD91CEB76
:10026000030306F1FF3080F01F81994240F21C81A8
:10027000023E63445B1AA4B2B3FBF8F008FB1033F0
:1002800044EA034400FB07F7A7420AD91CEB040425
:1002900000F1FF3380F00A81A74240F207816444F5
:1002A000023840EA0640E41B00261DB1D44000237A
:1002B000C5E900433146BDE8F0878B4209D9002DDE
:1002C00000F0EF800026C5E9000130463146BDE868
:1002D000F087B3FA83F6002E4AD18B4202D38242D2
:1002E00000F2F980841A61EB030301209E46002D81
:1002F000E0D0C5E9004EDDE702B9FFDEB2FA82F2D6
:10030000002A40F09280A1EB0C014FEA1C471FFA33
:100310008CFE0126200CB1FBF7F307FB131140EA1A
:1003200001410EFB03F0884208D91CEB010103F1E7
:10033000FF3802D2884200F2CB804346091AA4B2A9
:10034000B1FBF7F007FB101144EA01440EFB00FE7D
:10035000A64508D91CEB040400F1FF3102D2A645E2
:1003600000F2BB800846A4EB0E0440EA03409CE781
:10037000C6F12007B34022FA07FC4CEA030C20FA2E
:1003800007F401FA06F31C43F9404FEA1C4900FA4E
:1003900006F3B1FBF9F8200C1FFA8CFE09FB1811CB
:1003A00040EA014108FB0EF0884202FA06F20BD93E
:1003B0001CEB010108F1FF3A80F08880884240F28E
:1003C0008580A8F102086144091AA4B2B1FBF9F0D2
:1003D00009FB101144EA014100FB0EFE8E4508D9CD
:1003E0001CEB010100F1FF346CD28E456AD9023852
:1003F000614440EA0840A0FB0294A1EB0E01A14237
:10040000C846A64656D353D05DB1B3EB080261EBA4
:100410000E0101FA07F722FA06F3F1401F43C5E97E
:10042000007100263146BDE8F087C2F12003D840B4
:100430000CFA02FC21FA03F3914001434FEA1C47F6
:100440001FFA8CFEB3FBF7F007FB10360B0C43EAE8
:10045000064300FB0EF69E4204FA02F408D91CEB98
:10046000030300F1FF382FD29E422DD90238634496
:100470009B1B89B2B3FBF7F607FB163341EA034136
:1004800006FB0EF38B4208D91CEB010106F1FF3885
:1004900016D28B4214D9023E6144C91A46EA00467C
:1004A00038E72E46284605E70646E3E61846F8E60E
:1004B0004B45A9D2B9EB020864EB0C0E0138A3E757
:1004C0004646EAE7204694E74046D1E7D0467BE738
:1004D000023B614432E7304609E76444023842E7B0
:1004E000704700BF02E000F000F8FEE772B63A483D
:1004F00080F30888394880F3098839484EF6085156
:10050000CEF20001086040F20000CCF200004EF68E
:100510003471CEF200010860BFF34F8FBFF36F8FCD
:1005200040F20000C0F2F0004EF68851CEF2000119
:100530000860BFF34F8FBFF36F8F4FF00000E1EE05
:10054000100A4EF63C71CEF200010860062080F3DE
:100550001488BFF36F8F03F0A1F803F07DF803F068
:10056000C7F84FF055301F491B4A91423CBF41F834
:10057000040BFAE71C49194A91423CBF41F8040BAD
:10058000FAE71A491A4A1B4B9A423EBF51F8040B2C
:1005900042F8040BF8E700201749184A91423CBF83
:1005A00041F8040BFAE703F05BF803F0EFF8144CA2
:1005B000144DAC4203DA54F8041B8847F9E700F005
:1005C00041F8114C114DAC4203DA54F8041B884732
:1005D000F9E703F043B800000007002000230020E3
:1005E000000000080001002000070020603E000815
:1005F000002300201C230020202300208439002019
:10060000E0010008E0010008E0010008E001000846
:100610002DE9F04F2DED108AC1F80CD0C3689D462E
:10062000BDEC108ABDE8F08F002383F311882846C3
:10063000A047002002F0A8FCFEE702F02DFC00DF3E
:10064000FEE700002DE9F04102F052FF074602F0FC
:100650009FFF0546A8BB274B9F4232D001339F42E4
:1006600032D0254B27F0FF029A4231D1F8B200F088
:1006700043FAA84642F2107400F048FC00F042FA37
:10068000064648B354BB464635B11C4B9F4203D087
:1006900002F076FF00242646002002F033FF0EB160
:1006A00000F02EF800F054FC00F028FE00F02AFFC5
:1006B0000546B4B900F0ECFC4FF47A7002F06AFC25
:1006C000F7E7A8460024D7E704464FF00108D3E730
:1006D00080464FF47A74CFE70446D5E74FF47A7436
:1006E000D2E700F00FFF431BA342E3D900F008F864
:1006F000DCE700BF010007B0000008B0263A09B0EF
:100700001E4B1F4A10B51C461968013134D0043302
:100710009342F9D162681B4B9A422DD91A4B9B68C0
:1007200003F1006303F580339A4225D202F0FAFE0A
:1007300002F00CFF002000F0FBFD144B02201870AB
:1007400000F032FE124B1A6C00221A64196E1A66FF
:10075000196E596C5A64596E5A665B6E72B64FF0D8
:10076000E0232021C3F8084DD4E9003281F3118839
:100770009D4683F30888104710BD00BF00000108A4
:1007800020000108FFFF0008002300202023002094
:1007900000380240094A136849F2690099B21B0CFB
:1007A00000FB01331360064B186844F2506182B2BB
:1007B000000C01FB0200186080B270471823002073
:1007C0001423002010B500211022044600F008FE7A
:1007D000034B03CB206061601868A06010BD00BFB0
:1007E000107AFF1F2DE9F043204DBBB000F08AFEC8
:1007F000AB68C31AF92B32D906AFA8602B46282262
:100800000021384601F016FB05F10E0000F0E0FD76
:10081000002604465FFA80F905F10E08F3B2F100F4
:10082000994501F1280107D908EB0603082238464B
:1008300001F000FB0136F1E708230122CDE9023285
:1008400005340B4B0193A4B230230093CDE904741B
:1008500004A3D3E90023297B064801F003F93BB048
:10086000BDE8F08378F6339F93CACD8D60330020C6
:100870006D3300203C33002070B50D4614461E46F3
:1008800001F086F850B9022E10D1012C0ED112A31E
:10089000D3E90023C5E90023012007E0282C10D06C
:1008A00005D8012C09D0052C0FD0002070BD302CAC
:1008B000FBD10BA3D3E90023ECE70BA3D3E900237F
:1008C000E8E70BA3D3E90023E4E70BA3D3E9002374
:1008D000E0E700BFAFF30080401DA12026812A0B76
:1008E00078F6339F93CACD8D9E6AC421818A46EEE5
:1008F00026417272DF25D7B7F017304A39059E5668
:1009000013B504462346084620220021019001F039
:1009100091FA22790198032A234628BF032203F87B
:10092000042F2021022201F085FA62790198072A1A
:10093000234628BF072203F8052F2221032201F0B6
:1009400079FAA2790198072A234628BF072203F8DB
:10095000062F2521032201F06DFA019804F1080306
:100960001022282101F066FA382002B010BD0000E4
:100970002DE9F04FFFB01FAD0CAE40F2751280466E
:100980000F4620A80021296000F02AFD48220021FE
:10099000304600F025FD00F0B5FD554B4FF47A725E
:1009A000B0FBF2F0186093E80700012386E8070027
:1009B0000DF152003382FFF705FF41F20443338407
:1009C00006AB18464B4903F03DF91722306429461F
:1009D000304686F83C20FFF793FF10AB04460146F3
:1009E0000822284601F026FA0822A1180DF1410339
:1009F000284601F01FFA0DF14203082204F110010C
:100A0000284601F017FA11AB202204F118012846FC
:100A100001F010FA12AB402204F13801284601F02F
:100A200009FA14AB082204F17801284601F002FA11
:100A30000DF15103082204F18001284601F0FAF972
:100A400004F1880A0DF1520904F5847B4B465146A6
:100A5000082228460AF1080A01F0ECF9D34509F109
:100A60000109F3D119AB08225946284601F0E2F9F1
:100A700004F588744FF0000996F834304B450AD9D4
:100A8000B36B21464B440822284601F0D3F90834C1
:100A900009F10109F0E74FF0000996F83C304B45A9
:100AA00004EBC90108D9336C08224B44284601F0F5
:100AB000C1F909F10109F0E700230393BB7E02931A
:100AC000073107F119030193C1F3CF010123CDE9E8
:100AD00004510093F97E04A3D3E90023404600F0BB
:100AE000C1FF7FB0BDE8F08F9E6AC421818A46EEC7
:100AF00024230020543C0008014B1870704700BFAD
:100B000030230020F0B5334B1C7B85B034B1324B21
:100B10000E221A810024204605B0F0BD2F4A10682D
:100B2000516802AB03C308232D492E480DEB030285
:100B300003F066F8054630B9274B2B480A221A8184
:100B400000F09AFCE6E70169B1F5E02F06D9224BE7
:100B500026480B221A8100F08FFCDCE7438B40F221
:100B60001442934207D01C490C20088119462048A2
:100B700000F082FCCFE71F4A024402F110039942C1
:100B800004D2154B1C4810221A81E4E710398E1A42
:100B90002046144900F0BAFC3246074605F1180118
:100BA000204600F0B3FCAB689F4202D1EB6898424C
:100BB0000AD0094B0D221A810090D5E902123B465A
:100BC0000E4800F059FCA5E70D4800F055FC012443
:100BD000A1E700BF6033002024230020FD3C000873
:100BE000DCFF0600000001086C3C0008783C0008AF
:100BF0008A3C00080800FFF7A83C0008C53C000834
:100C0000EE3C00082DE9F04FADB006AF80460C4633
:100C100000F0BEFE054600285AD1237E022B1BD1D0
:100C2000E38A012B18D100F06DFC0646FFF7B2FDF8
:100C300003464FF4C870DFF8D092B3FBF0F206F52C
:100C4000167602FB103316FA83F3C9F80030E37E00
:100C500033B9A84B00221A709C37BD46BDE8F08F0F
:100C6000A38AEEB2013BB34205F101050BD93B1D4E
:100C70001E44E90000960023082201F0F8012046F6
:100C800000F09CFFECE707F11400FFF79BFD3246F4
:100C900007F11401381D02F0A3FF0028D9D10F2E4F
:100CA00008D8944B1E70D9F80030A3F51673C9F814
:100CB0000030D1E7FB1CF870014600930722034681
:100CC000204600F07BFFF978404600F059FEC3E76C
:100CD000E38A282B26D010D8012B1ED0052BBBD1A0
:100CE000BFF34F8F8449854BCA6802F4E062134317
:100CF000CB60BFF34F8F00BFFDE7302BACD1637EDD
:100D00007F4D01336A7BDBB29342E94603D1E27E39
:100D10002B7B9A4265D0CD469EE721464046FFF7A1
:100D200027FE99E7A38A013B9BB2C92B94D8744D47
:100D30002E7B26BB05F10C03009308223346314677
:100D4000204600F03BFF731CF2B2D9001E46A38A76
:100D5000013B9A4205DA0E322A440092002308220F
:100D6000EEE700230022C5E900230023AB6085F8ED
:100D7000D730C5F8D8302B7B0BB9E37E2B73002519
:100D800007F114093B1D082229464846C7E90155C9
:100D9000FD6001F04FF83B7A05F1010AAB424FEAE2
:100DA000CA0608D9FB6808222B443146484601F0A0
:100DB00041F85546EFE7C6F3CF06E17ECDE904964C
:100DC00000230393A37E02931934282300930194F4
:100DD00046A3D3E90023404600F044FEFFF702FD9E
:100DE0003AE74FF0000807F11403A7F81480102227
:100DF000009341460123204600F0E0FEA68A023E11
:100E0000B6B2F31C9B109B000733DB08A9EBC303AE
:100E10009D460DF1180A1FFA88F34FEAC801B34244
:100E200001F110010AD20AEB080300930822002303
:100E3000204600F0C3FE08F10108ECE795F8D70062
:100E400000F080FAD5F8D83004461BB995F8D700E1
:100E500000F088FAD5F8D83033449C4204D295F893
:100E6000D700013000F07EFA4FEA960B4FF00008F1
:100E70001FFA88F18B45D5E9003209D90AEB8801C0
:100E800003EB8800012200F0B3FA08F10108EFE754
:100E9000F31842F10002C5E90032D5F8D83095F8D0
:100EA000D70006EB0308C5F8D88000F04BFA804560
:100EB00009D395F8D730D5F8D8000133001B85F851
:100EC000D730C5F8D800FF2E08D800232B7300F0C8
:100ED0005BFAFFF717FE08B1FFF712FC2B68094A0F
:100EE0009B0A013313810023AB6014E72641727221
:100EF000DF25D7B73533002000ED00E00400FA0508
:100F000060330020242300203833002008B54FF040
:100F100000530B4A196891420AD10A4A597D11704F
:100F200009481B7D03730949C9220E3000F046FAB7
:100F3000BDE80840E02200214FF0005000F050BA18
:100F40009AAD44C5302300206033002016000020F5
:100F50002DE9FF41434C02236371002302931825BE
:100F60000A23581EB5FBF3F67343D3F11802C1B23E
:100F70003ED002280346F4D19DF80B303A493B4855
:100F80005A1E9DF80A30013B1B0443EA0253BDF888
:100F90000820013A13434B6001F09EFC00230193AB
:100FA000334B344900933448344B4FF4805200F0B3
:100FB000C1FC334B197811B12F4800F0E1FC00F06F
:100FC000A1FA0546FFF7E6FB4FF4C873B0FBF3F256
:100FD00002FB130305F5167010FA83F0294B186015
:100FE00002F0D6FA08B10F23238104B0BDE8F081E6
:100FF000C1EBC107FB1C4FEAE30EC3F3C703A1EB30
:10100000030C0EF101084FF47A705FFA8CF50EFBB9
:10101000000058FA8CFCB0FBFCF0B0F5617F07D9FA
:101020007B1EC3F3C703C91ACDB2591E0F2916D8A8
:101030006A1E072A8CBF00220122591901FB066093
:101040001149B1FBF0F11148814295D1002A93D0AA
:10105000ADF808608DF80A308DF80B508CE7134618
:10106000EBE700BF242300200C230020783400206D
:1010700079080008342300203C330020050C0008C8
:10108000302300203833002000366E0140420F002C
:101090002DE9F04F91A7D7E900670FF24829D9E968
:1010A0000089874D93B0DFF844B2864C284600F0A3
:1010B0003DFD0DF1300A079070B31022002150461B
:1010C00000F08EF9079B197B4FF0000261F30302D9
:1010D0008DF83020586899680EAA03C21B680D9AD3
:1010E00063F31C029DF830300D9243F020038DF81D
:1010F0003030002352461946584601F0FDFB079058
:1011000028B9284600F016FD079B2370CEE7237808
:10111000072B3CD80133237018220021504600F0E1
:101120005FF9DFF8C8B1684C0023194652465846AB
:1011300001F00AFC014670BB102208A800F050F92B
:10114000636983F02003636100F0DEF90B4612A9A6
:10115000024611E903000DF1240C8CE803009DF810
:101160003410C1F3030089064CBF0E99BDF838C096
:101170008DF82C0046BFC1F31C0C4CF00041CCF3A1
:101180000A010891284608A900F09CFECCE72846F1
:1011900000F0D0FCC0E7284600F0FAFB0446002827
:1011A00048D1DFF84CB100F0ADF9DBF800309842DF
:1011B00040D300F0A7F90790FFF7ECFA079A8DF8F3
:1011C000204003464FF4C87002F51672B3FBF0F1ED
:1011D00001FB103312FA83F3CBF80030DFF814B1BF
:1011E0009BF8001011B901238DF82030504607916B
:1011F000FFF7E8FA0799C1F11004E4B2062C28BF02
:101200000624224651440DF1210000F0D7F808AB26
:1012100003931823029301342C4B0193E4B201236E
:10122000009304943B463246284600F0B3FB00236B
:101230008BF8003000F066F9254A264C1368C31A73
:10124000B3F57A7F31D3106000F05EF902460B46A9
:10125000284600F079FC284600F09AFB28B3237B4F
:10126000DFF894B0002B14BF032302238BF8053062
:1012700000F048F94FF47A735146B0FBF3F0CBF825
:1012800000005846FFF73CFB182307300293124B2F
:101290000193C0F3CF0040F25513CDE903A00093B2
:1012A00042464B46284600F075FB237B2BB1FFF7E7
:1012B00099FA237B002B7FF4F6AE13B0BDE8F08FD4
:1012C0003C3300204534002000000240343300202D
:1012D000403400206033002044340020401DA12011
:1012E00026812A0BF1C6A7C1D068080F78340020E8
:1012F00038330020353300202423002070B501F05E
:10130000ABFF094E094D30800024286833888342A2
:1013100008D901F09BFF2B6804440133B4F5803FEA
:101320002B60F2D370BD00BF74340020483400201D
:1013300002F042B800F10060920000F5803001F048
:10134000D1BF0000054B1A68054B1B889B1A8342CE
:1013500002D9104401F07ABF0020704748340020C1
:101360007434002038B5074D04462868204401F045
:1013700075FF28B928682044BDE8384001F086BFD1
:1013800038BD00BF48340020064991F8243033B1FD
:101390000023086A81F824300822FFF7CBBF012020
:1013A000704700BF4C340020022802BF024B4FF4AC
:1013B00000129A61704700BF0000024010B5002380
:1013C000934203D0CC5CC4540133F9E710BD000054
:1013D00003460246D01A12F9011B0029FAD17047C0
:1013E00002440346934202D003F8011BFAE7704718
:1013F0002DE9F8431F4D144695F8242007468846EA
:1014000052BBDFF870909CB395F824302BB92022A2
:10141000FF2148462F62FFF7E3FF95F82400C0F153
:101420000802A24228BF2246D6B24146920005EBEE
:101430008000FFF7C3FF95F82430A41B1E44F6B2CA
:10144000082E17449044E4B285F82460DBD1FFF7FE
:101450009BFF0028D7D108E02B6A03EB820383426D
:10146000CFD0FFF791FF0028CBD10020BDE8F88353
:101470000120FBE74C3400200FB4002004B070477B
:10148000FEE7000000B59BB0EFF3098168226846D3
:10149000FFF794FFEFF30583044B9A6BDA6A9A6ABD
:1014A0009A6A9A6A9A6A9A6A9B6AFEE700ED00E075
:1014B00000B59BB0EFF3098168226846FFF77EFF15
:1014C000EFF30583044B9A6B9A6A9A6A9A6A9A6A4E
:1014D0009A6A9B6AFEE700BF00ED00E000B59BB092
:1014E000EFF3098168226846FFF768FFEFF3058391
:1014F000034B5A6B9A6A9A6A9A6A9A6A9B6AFEE7DF
:1015000000ED00E001F092BF01F06ABF30B5094D77
:101510000A4491420DD011F8013B5840082340F392
:101520000004013B2C4013F0FF0384EA5000F6D185
:10153000EFE730BD2083B8ED2DE9F041C56915B95D
:10154000C161BDE8F0814B6823F06047C3F38A4670
:101550004FEAD37EC3F3807816EA230638BF3E46AF
:10156000AC462B465A68BEEBD27F22F060440AD0CC
:10157000002A18DAA40CB44217D19D420FD10D6095
:10158000DEE71346EEE7A74207D102F08044C2F33C
:10159000807242450BD054B1EFE708D2EDE7CCF8AA
:1015A00000100B60CDE7B44201D0B442E5D81A6810
:1015B0009C46002AE5D11960C3E700002DE9F047F9
:1015C000089D01F007044FEAD508224405F00705FD
:1015D00000EBD1004FF47F49944201D1BDE8F08780
:1015E00004F0070705F0070A57453E4638BF564640
:1015F000C6F10806111B8E4228BF0E46E10808EB13
:10160000D50E415C13F80EC0B94029FA06F721FA4D
:101610000AF1FFB28CEA010147FA0AF739408CEA75
:10162000010C03F80EC034443544D5E780EA0120AC
:10163000082341F2210201B24000002980B203F1E7
:10164000FF33B8BF504013F0FF03F4D170470000E0
:1016500038B50C468D18A54200D138BD14F8011BD1
:10166000FFF7E4FFF7E7000002684AB11368036080
:10167000C388018901339BB29942C38038BF03817B
:101680001046704770B588B0202204460D46684663
:101690000021FFF7A5FE20460495FFF7E5FF02466F
:1016A00058B16B46054608AE1C4603CCB4422860D0
:1016B0006960234605F10805F6D1104608B070BDF3
:1016C00010B54B6823B9CA8A63F30902CA8210BDF8
:1016D000C4681A681C60C360438A013B43824A6045
:1016E000EFE700002DE9F84F1D46CB8A0F46C3F304
:1016F00009010629814692460B4630D00020AAB245
:1017000007F119049EB2052E1FFA80F80FD89045F4
:1017100003F1010306D3FB8A0A4462F30903FB8247
:1017200001201AE01AF80060E6540130EAE790451B
:10173000F1D2A1F1060B1C237C68BBFBF3F203FB87
:1017400012BB1FFA8BF6002C45D14846FFF78CFFE1
:10175000044638B978606FF00200BDE8F88F4FF0AA
:101760000008E6E7002606607860ADB24FF0000B97
:10177000454510D90AEB0803221D13F8011B9155AA
:10178000B1B208F101081B291FFA88F82BD0454592
:1017900006F10106F1D8FB8AC3F30902154465F38B
:1017A0000903BCE7013292B21C462368002BF9D131
:1017B000AB1F0B441C21B3FBF1F301339BB29A42E4
:1017C000D3D2BBF1000FD0D14846FFF74DFF20B96F
:1017D000C4F800B0BFE70122E7E7C0F800B05E46FA
:1017E00020600446C1E74545D5D94846FFF73CFF90
:1017F00008B92060AFE7C0F800B0002620600446BA
:10180000B6E700002DE9F04F2DED028B83B0CDE956
:101810000013BDF83C4080469246002A00F08780C5
:101820002CB10E9B002B00F08280072C2BD808F1E6
:101830000C00FFF719FF054638B96FF0020528467E
:1018400003B0BDEC028BBDE8F08F14220021FFF73E
:10185000C7FD22460E9905F10800FFF7AFFD631C96
:101860002B749AF800302C4403F01F0363F03F03FD
:101870002372009B43F00041696040462946FFF710
:101880005BFE0125DBE700F10C034FF0000908EED9
:10189000103A4FF0800B4E464D4618EE100AFFF7F7
:1018A000E3FE07460028C8D014220021FFF798FD68
:1018B000002E3AD1019B3B8102220E9B02F10801CE
:1018C00003EB060C57FA81F11046B44202F1010213
:1018D000D2B201D8024607E01CF8010B01F8010B57
:1018E0000136062AB6B2EFD99AF8001001F01F01AE
:1018F000B44208BF4FF0400BB81841EA49114BEA17
:1019000001030372009B013243F000437B603A7491
:1019100039464046FFF710FE0135B4422DB289F03A
:1019200001094FF0000BB8D189E70022C5E76FF03D
:10193000010584E7F8B515460E4624220021044629
:101940001F46FFF74DFD069B6360B5F5001F079B23
:10195000A76034BF6A094FF6FF72236204F10C00DE
:1019600097B200239A4205D800230360278263823E
:10197000A382F8BD0660013330462036F2E700004E
:1019800003781BB94BB2002BC8BF01707047000031
:10199000007870472DE9F74FDDF83C90BDF83050E6
:1019A0000D9E9DF83840BDF84070804692469B469B
:1019B000B9F1000F01D1002F51D11F2C4FD898F849
:1019C0000000B0B9072F47D835F0030347D13A4696
:1019D00049464FF6FF70FFF73BFE20F001002D0255
:1019E000400445EA0464400C44EA40244FF6FF7387
:1019F00021E040EA0520072F40EA0464F6D90025DB
:101A00004FF6FF73C5F12000A5F120022AFA05F177
:101A10000BFA00F001432BFA02F211431846C9B247
:101A2000FFF704FE0835402D0346EBD13A46494600
:101A3000FFF70EFE0346CDE90097324621464046A9
:101A4000FFF7E0FE33780133DBB21F2B88BF0023A2
:101A5000337003B0BDE8F08F6FF00300F9E76FF06B
:101A60000100F6E72DE9F04F85B09246DDF8488099
:101A70000F9D9DF840209DF84490BDF84C7006469F
:101A80009B46B8F1000F01D1002F48D11F2A46D83C
:101A90003378002B46D00C0244EA02649DF83810DB
:101AA00044EAC93444EA01441C43072F44F080044B
:101AB00032D900234FF6FF72C3F1200CA3F12000AE
:101AC0002AFA03F10BFA0CFC41EA0C012BFA00F0A4
:101AD0000143C9B210460393FFF7A8FD039B0833E7
:101AE000402B0246E8D13A464146FFF7B1FD034696
:101AF000CDE900872A4621463046FFF783FEB9F13B
:101B0000010F06D12B780133DBB21F2B88BF0023D6
:101B10002B7005B0BDE8F08F4FF6FF73E8E76FF06C
:101B20000100F6E76FF00300F3E70000C06900B1C1
:101B300004307047C3691A68C261C2681A60C36022
:101B4000438A013B438270472DE9F041D0F8188069
:101B5000194E14461D464146002709B9BDE8F081DB
:101B6000D1E90223A21A65EB0303964277EB030344
:101B70001ED283698B420DD1FFF7A2FD83691B68DA
:101B80008361C3680B60438AC1608169013B438202
:101B90008846E2E7FFF794FD0B68C8F80030C36899
:101BA0000B60438AC160013B4382D8F80010D4E740
:101BB00088460968D1E700BF80841E002DE9F04FF8
:101BC0008BB00D46DDF8509014469B4680460028A9
:101BD00000F01981B9F1000F00F01581531E3F2B61
:101BE00000F21181012A03D1BBF1000F40F00B81FB
:101BF0000023CDE90833B8F81430B5EBC30F4FEA32
:101C0000C30703D300200BB0BDE8F08F2B199F4210
:101C1000D8F80C303ABF7F1BFFB227461BB9D8F863
:101C20001030002B7AD02F2D4ED8C5F13006B74298
:101C30004FF000032CBFF6B23E4600932946D8F879
:101C4000080008AB3246FFF7B9FCA7EB060A35449B
:101C50005FFA8AFAB8F8143003F10053063BDB0050
:101C60000493D8F80C3003933021039B13B1BAF1DD
:101C7000000F2CD1D8F8100040B1BAF1000F05D0F8
:101C8000009608AB5246691AFFF798FC38B2002F4D
:101C9000B8D066070AD00AAB03EBD401624211F850
:101CA000083C02F00702134101F8083C082C3CD91B
:101CB000102C40F2B580202C40F2B780BBF1000F11
:101CC00000F09C80082334E0BA460026C2E7049B5B
:101CD000E02B28BFE02306930B44AB42059314D9B5
:101CE0005A1B03980096924534BF5246D2B2691AE5
:101CF00008AB04300792FFF761FC079A1644AAEB81
:101D0000020A1544F6B25FFA8AFA049B069A05990C
:101D10009B1A0493039B1B680393A6E70093D8F8D0
:101D2000080008AB3A462946AEE7BBF1000F13D0D6
:101D30000123B4EBC30F6CD0082C12D89DF82030CF
:101D4000621E23FA02F2D50706D54FF0FF3202FADF
:101D500004F423438DF820309DF8203089F80030BA
:101D600051E7102C12D8BDF82030621E23FA02F27F
:101D7000D10706D54FF0FF3202FA04F42343ADF841
:101D80002030BDF82030A9F800303CE7202C0FD8D7
:101D90000899631E21FA03F3DA0705D54FF0FF32E5
:101DA00002FA04F40C430894089BC9F800302AE7AF
:101DB000402C2BD0DDE90865611EC4F12102A4F19D
:101DC000210326FA01F105FA02F225FA03F3114381
:101DD0001943CB0712D50122A4F12003C4F120013D
:101DE00002FA03F322FA01F1A240524243EA01034C
:101DF00063EB430332432B43CDE90823DDE908239A
:101E0000C9E90023FFE66FF00100FCE66FF008006F
:101E1000F9E6082CA0D9102CB3D9202CEED8C3E7B2
:101E2000BBF1000FADD0022383E7BBF1000FBBD0A5
:101E300004237EE730B5012A144638BF0124402C24
:101E400085B028BF40240025012ACDE9025518D8C5
:101E50001B788DF8083063070AD004AB03EBD40578
:101E6000624215F8083C02F00702934005F8083C6E
:101E7000009103462246002102A8FFF79FFB05B010
:101E800030BD082AE4D9102A03D81B88ADF80830E1
:101E9000E1E7202A8DBFD3E900231B680293CDE937
:101EA0000223D8E710B5CB681BB98B600B618B821E
:101EB00010BDC4681A681C60C360438A013B43823A
:101EC000CA60F0E72DE9F04FD1F8008093B018F028
:101ED000800FCDE90323C8F3C01219BFC8F3C03B7C
:101EE000C8F306264FF0020B1646B8F1000F044661
:101EF0000D4680F2C58118F0C043059340F0C081C3
:101F00000B7B002B00F0BC81BBF1020F03D00178EA
:101F1000B14240F0B88108F07F0106916AB3C8F37E
:101F2000074A2B44069A93F80390760646EA0B4636
:101F300046EA82465FEAD91346EA0A06079300F0AA
:101F4000908000220023CDE90A23069B0093676856
:101F50005B4652460AA92046B84700287ED0A769AA
:101F60009FB9314604F10C00FFF78CFB0746E0B93E
:101F70006FF0020013B0BDE8F08FC8F30F2A18F01D
:101F80007F0F08BF0AF0030ACBE73B699E420DD0E2
:101F90003F68002FF9D1314604F10C00FFF772FBC6
:101FA00007460028E4D0A3693B60A761DDE90A2366
:101FB00000264FF6FF70C6F1200E22FA06F103FA52
:101FC0000EFEA6F1200C23FA0CFC41EA0E0141EAB8
:101FD0000C01C9B2083609920893FFF727FB402E7F
:101FE000DDE90832E7D1B882FB7D09F01F06C3F3B3
:101FF00084039B1BD7E9022198B2002BBCBF00F1E0
:1020000020031BB252EA0100C8F304680FD0039802
:10201000821A049860EB0101A14890424FF000023F
:102020008A4104D3079A002A55D0012B23DDFA7D7B
:102030004FEA890302F0030203F07C031343FB75AC
:1020400039462046FFF73CFB079BA3B9FB7DC3F352
:102050008402013262F38603FB7504E06FF00B002B
:1020600088E7A76917B96FF00C0083E73B699E42C8
:10207000BAD03F68F6E719F0400F2CD0039BBB6045
:10208000049BFB60142200210DA8FFF7A9F9039B14
:102090000A93049B0B932B1D0C932B7BADF83EA056
:1020A000013BDBB2ADF83C30069B8DF843308DF838
:1020B00040B0A3688DF841608DF842800AA920469F
:1020C0009847FB7DC3F38403013303F01F039B0296
:1020D000FB8200204EE7FB7DC9F34012B2EBD31F19
:1020E00040F0D480C3F38403B34240F0D280079918
:1020F0002B7B4FEA9912002934D0D20741D4032B0D
:1021000040F2CA80039BBB60049BFB602B7BAE1D2F
:10211000033BDBB23246394604F10C00FFF7E2FA2A
:1021200000280DDA20463946FFF7CAFAFB7DC3F3D3
:102130008403013303F01F039B02FB82032019E792
:10214000AB883B832A7B033AB88AD2B23146FFF789
:102150007FFAFB7DB882DA43C2F3C01262F3C71381
:10216000FB75B6E76AB92E1D013BDBB23246394634
:1021700004F10C00FFF7B6FA0028D3DB2A7B013A02
:10218000E2E7F98AC1F30901013B0529DAB253D824
:10219000281D002307F11A0C9A4208D910F801EB08
:1021A0000CF801E0013101330629DBB2F4D10399C7
:1021B0000A9104990B91934207F11A010C9138BFCF
:1021C000043379680D9134BF55FA83F300230E93DD
:1021D000FB8AADF83EA0C3F309031A44069B8DF8B1
:1021E00043300023ADF83C208DF840B08DF84160BD
:1021F0008DF842807B602A7BB88A013A291DFFF75F
:1022000027FA3B8BB882834203D1A3680AA92046F0
:10221000984720460AA9FFF745FEFB7DB88AC3F31D
:102220008403013303F01F039B02FB823B8B984224
:1022300014BF112000209DE67B68002BB7D006203C
:1022400001E01C306346D3F800C0BCF1000FF8D1A8
:10225000091A081D05F1040C00EB030905989DF807
:10226000143001EB000EBEF11B0FA0D89A429ED98C
:102270001CF8013B09F8013B059B01330593EDE791
:102280006FF0090076E66FF00A0073E66FF00D005C
:1022900070E66FF00E006DE66FF00F006AE600BFAB
:1022A00080841E00404BF0B51C6C404E44F000741E
:1022B0001C641D6E45F000751D661B6E3C4B9B6AD1
:1022C000D3F80052354045F00105C3F80052D3F869
:1022D0000042344044EA002040F00100C3F800020C
:1022E000002952D00020C3F81C020546C3F804029E
:1022F000C3F80C02C3F8140203EBC00401301C281D
:10230000C4F84052C4F84452F6D100254FF0010CF5
:1023100096781488F70748BFD3F804720CFA04F0D3
:1023200044BF0743C3F80472B70742BFD3F80C7227
:102330000743C3F80C72760742BFD3F81462064312
:10234000C3F8146203EBC4045668C4F8406296688C
:10235000C4F84462D3F81C4201352043A942C3F8B3
:102360001C0202F10C02D3D1D3F8002222F00102A8
:10237000C3F800220C4B1A6C22F000721A641A6E19
:1023800022F000721A661B6EF0BD0122C3F84012E3
:10239000C3F84412C3F80412C3F81412C3F80C2291
:1023A000C3F81C22E0E700BF003802400000FFFF36
:1023B00078340020184A916A08B58B688B6013F056
:1023C000010104D013F00C0F18BF4FF48031D80571
:1023D00006D513F4406F14BF41F4003141F00201FF
:1023E000D80306D513F4402F14BF41F4802141F0E7
:1023F0000401D3690BB108489847202383F311885F
:102400000648002100F0EEFD002383F31188BDE8AB
:10241000084001F0F7B800BF783400208034002075
:1024200038B5124CA36ADD68AA0712D05A6922F0A7
:1024300002025A61A36913B1012120469847202363
:1024400083F311880A48002100F0CCFD002383F3B8
:102450001188EB0606D5A36A1021D960236A0BB157
:1024600002489847BDE8384001F0CCB878340020E5
:102470008834002038B5124CA36A1D69AA0712D00F
:102480005A6922F010025A61A36913B10221204651
:102490009847202383F311880A48002100F0A2FD09
:1024A000002383F31188EB0606D5A36A1021196176
:1024B000236A0BB102489847BDE8384001F0A2B842
:1024C000783400208834002038B50F4CA36A5D684A
:1024D0005D602A070AD5042222701A6822F00202DF
:1024E0001A60636A13B10021204698476B0706D52E
:1024F000A36A9969236A13B1034809049847BDE8A0
:10250000384001F07FB800BF7834002010B50E4C81
:10251000204600F0CFF90D4BA3620B21132000F0F1
:10252000B1F90B21142000F0ADF90B21152000F0BA
:10253000A9F90B21162000F0A5F90022BDE81040F2
:1025400011460E20FFF7AEBE783400200064004034
:10255000114B984210B5044609D1104B1A6C42F049
:1025600000721A641A6E42F000721A661B6EA36A39
:1025700001221A60A36A5A68D20707D562685168B7
:102580001268D9611A60064A5A6110BD01210820FB
:1025900000F01EFCEEE700BF783400200038024057
:1025A0005B87010003291AD8DFE801F0020A0F1443
:1025B000836A9B6813F0E05F14BF0120002070471E
:1025C000836A9868C0F380607047836A9868C0F334
:1025D000C0607047836A9868C0F30070704700203D
:1025E0007047000010B5032925D8DFE801F0022567
:1025F000292D836A9968C1F30161183103EB011336
:10260000107884064CBF54689488C0F300114FEAD8
:10261000410148BF41EAC40100F00F004CBF41F046
:10262000040141EA4451586041F001019068D268C8
:102630009860DA60196010BD836A03F5C073DFE744
:10264000836A03F5C873DBE7836A03F5D073D7E7C2
:1026500001290AD002290FD081B9836ADA6892076A
:1026600001D1186903E001207047836AD86810F02F
:10267000030018BF01207047836AF2E7002070470B
:1026800010B539B9836AD96889071BD11B699C07C2
:1026900004D110BD012915D00229FAD1816AD1F8DF
:1026A000C031D1F8C441D1F8C8011061D1F8CC01D2
:1026B0005061202008610869800717D1486940F0FF
:1026C000100012E0816AD1F8B031D1F8B441D1F8EC
:1026D000B8011061D1F8BC0150612020C860C86801
:1026E000800703D1486940F002004861C3F340000D
:1026F000C3F38001000140EA4111107920F030005D
:102700000143117189064BBF91681189DB085B0D8C
:102710004CBF63F31C0163F30A01137948BF916056
:1027200064F3030313714FEA14234FEA144458BFB0
:10273000118113705480ACE7024AD36843F0C003A0
:10274000D360704700140140044B5A6810439A68E4
:1027500058600AB1181D1047704700BFA43400200C
:102760002DE9F0413C4ED6F85C52EF682B68DA0553
:102770009CB20CD5202383F311884FF40070FFF72F
:10278000E3FF6FF480732B60002383F31188202311
:1027900083F31188DFF8C08014F02F0339D183F35D
:1027A0001188380613D5210611D5202383F311880B
:1027B0002A4800F001FA00284CDA0820FFF7C4FF8D
:1027C0004FF67F733B40EB60002383F311887A065A
:1027D00015D5630613D5202383F31188D6E9132377
:1027E0009A4209D1336C3BB127F040073F041020D7
:1027F0003F0CFFF7A9FFEF60002383F31188D6F8A1
:102800006422D3680BB110699847BDE8F04100F02D
:10281000F9BE230712D014F0080F0CBF002080204F
:10282000E10748BF40F02000A20748BF40F0400049
:10283000630748BF40F48070FFF786FFA4066B680B
:1028400005D596F860124046194000F057FA2C68FA
:10285000A4B2A1E76860B7E7A4340020DC3400200C
:1028600010B5054C054A0021204600F025FA044B1E
:10287000C4F85C3210BD00BFA43400203927000822
:102880000014014000F1604303F561430901C9B23E
:1028900083F80013012200F01F039A4043099B00B4
:1028A00003F1604303F56143C3F880211A60704768
:1028B000FFF72CBE012300F10802C0E902220370D9
:1028C00000F110020023C0E90422C0E90633C0E988
:1028D000083343607047000010B52023044683F39B
:1028E0001188022303704160FFF732FE0423237036
:1028F000002383F3118810BD2DE9F0411F460446E3
:102900000D461646202383F3118800F1080823782A
:10291000052B0DD029462046FFF744FE40B1204646
:1029200032462946FFF75EFE002080F3118808E05A
:102930003946404600F03AFB0028E8D0002383F3F4
:102940001188BDE8F08100002DE9F0411F460446E2
:102950000D461646202383F3118800F110082378D2
:10296000052B0DD029462046FFF772FE40B12046C8
:1029700032462946FFF784FE002080F3118808E0E4
:102980003946404600F012FB0028E8D0002383F3CC
:102990001188BDE8F0810000F8B515468268066927
:1029A000AA420B46816938BF8568761AB54204464B
:1029B0000BD218462A46FEF701FDA3692B44A361FA
:1029C000A3685B1BA3602846F8BD0CD918463246A5
:1029D000FEF7F4FCAF1BE1683A463044FEF7EEFC2C
:1029E000E3683B44EBE718462A46FEF7E7FCE3685A
:1029F000E5E7000083689342F7B51546044638BF03
:102A00008568D0E90460361AB5420BD22A46FEF733
:102A1000D5FC63692B446361A36828465B1BA360F4
:102A200003B0F0BD0DD932460191FEF7C7FC019904
:102A3000E068AF1B3A463144FEF7C0FCE3683B4414
:102A4000E9E72A46FEF7BAFCE368E4E710B50A4472
:102A50000024C361029B8460C0E90000C0E9051145
:102A6000C1600261036210BD08B5D0E9053293422E
:102A700001D1826882B98268013282605A1C426147
:102A80001970D0E904329A4224BFC368436100211F
:102A900000F09CFA002008BD4FF0FF30FBE700007B
:102AA00070B5202304460E4683F31188A568A5B1AE
:102AB000A368A269013BA360531CA3611578226936
:102AC000934224BFE368A361E3690BB120469847B2
:102AD000002383F31188284607E03146204600F0A2
:102AE00065FA0028E2DA85F3118870BD2DE9F74F09
:102AF00004460E4617469846D0F81C904FF0200A20
:102B00008AF311884FF0000B154665B12A4631460D
:102B10002046FFF741FF034660B94146204600F0DA
:102B200045FA0028F1D0002383F31188781B03B005
:102B3000BDE8F08FB9F1000F03D001902046C847DF
:102B4000019B8BF31188ED1A1E448AF31188DCE790
:102B5000C0E90511C160C3611144009B8260C0E9F6
:102B60000000016103627047F8B504460D46164641
:102B7000202383F31188A768A7B1A368013BA36052
:102B800063695A1C62611D70D4E904329A4224BF01
:102B9000E3686361E3690BB120469847002080F346
:102BA000118807E03146204600F000FA0028E2DAFA
:102BB00087F31188F8BD0000D0E905239A4210B5CB
:102BC00001D182687AB98268013282605A1C8261BE
:102BD0001C7803699A4224BFC3688361002100F016
:102BE000F5F9204610BD4FF0FF30FBE72DE9F74F18
:102BF00004460E4617469846D0F81C904FF0200A1F
:102C00008AF311884FF0000B154665B12A4631460C
:102C10002046FFF7EFFE034660B94146204600F02C
:102C2000C5F90028F1D0002383F31188781B03B085
:102C3000BDE8F08FB9F1000F03D001902046C847DE
:102C4000019B8BF31188ED1A1E448AF31188DCE78F
:102C5000026843681143016003B1184770470000E0
:102C60001430FFF743BF00004FF0FF331430FFF77D
:102C70003DBF00003830FFF7B9BF00004FF0FF3311
:102C80003830FFF7B3BF00001430FFF709BF000072
:102C90004FF0FF311430FFF703BF00003830FFF76B
:102CA00063BF00004FF0FF323830FFF75DBF000018
:102CB00000207047FFF7D4BD37B515460E4A0260B5
:102CC00000224260C0E902220122044602740B463F
:102CD000009000F15C014FF480721430FFF7B6FEF3
:102CE00000942B464FF4807204F5AE7104F1380065
:102CF000FFF72EFF03B030BD083D000838B5C369AB
:102D000004460D461BB904210844FFF7A1FF2946DC
:102D100004F11400FFF7A8FE002806DA201D4FF486
:102D20008061BDE83840FFF793BF38BD024B0022F9
:102D3000C3E900339A6070470C3700200023037406
:102D40008268054B1B6899689142FBD25A68036000
:102D500042601060586070470C37002008B520238F
:102D600083F31188037C032B05D0042B0DD02BB9E2
:102D700083F3118808BD436900221A604FF0FF33C6
:102D80004361FFF7DBFF0023F2E7D0E90032136075
:102D90005A60F3E7002303748268054B1B68996847
:102DA0009142FBD85A6803604260106058607047D7
:102DB0000C370020054B19690874186802681A60FE
:102DC0005360186101230374FDF722BC0C37002007
:102DD00030B54B1C0B4D87B0044610D02B690A4A06
:102DE00001A800F01BF92046FFF7E4FF049B13B194
:102DF00001A800F04FF92B69586907B030BDFFF703
:102E0000D9FFF8E70C3700205D2D000838B50C4DD0
:102E100041612B6981689A689142044603D8BDE8F4
:102E20003840FFF78BBF1846FFF7B4FF01232C6132
:102E3000014623742046BDE83840FDF7E9BB00BFDA
:102E40000C370020044B1A681B6990689B689842F5
:102E500094BF0020012070470C37002010B5084CAB
:102E6000236820691A6822605460012223611A7461
:102E7000FFF790FF01462069BDE81040FDF7C8BB91
:102E80000C37002008B5FFF7DDFF18B1BDE808409A
:102E9000FFF7E4BF08BD0000FFF7E0BFFEE700005A
:102EA00010B50C4CFFF742FF00F0AAF80A49802247
:102EB000204600F031F8012344F8180C037400F0A8
:102EC0007DFB002383F3118862B60448BDE81040FF
:102ED00000F042B834370020303D0008403D000883
:102EE00000F012B9EFF3118020B9EFF3058320222F
:102EF00082F311887047000010B530B9EFF30584F4
:102F0000C4F3080414B180F3118810BDFFF7BAFFB1
:102F100084F31188F9E70000826002220282704780
:102F20008368A3F17C0243F80C2C026943F83C2C23
:102F3000426943F8382C074A43F81C2CC26843F80E
:102F4000102C022203F8082C002203F8072CA3F10E
:102F5000180070472906000810B5202383F3118854
:102F6000FFF7DEFF00210446FFF750FF002383F345
:102F70001188204610BD0000024B1B6958610F20CC
:102F8000FFF718BF0C370020202383F31188FFF7C9
:102F9000F3BF000008B50146202383F31188082001
:102FA000FFF716FF002383F3118808BD49B1064BD4
:102FB00042681B6918605A60136043600420FFF781
:102FC00007BF4FF0FF3070470C370020036898426E
:102FD00006D01A680260506059611846FFF7AEBE0D
:102FE0007047000038B504460D462068844200D181
:102FF00038BD036823605C604561FFF79FFEF4E71E
:10300000054B03F11402C3E905224FF0FF31002202
:10301000C3E90712704700BF0C37002070B51C4E83
:10302000C0E9032305460C4600F04EFB334653F837
:10303000142F9A420DD13062C5E901242A600A2C6E
:103040002CBF00190A30C6E90555BDE8704000F0F4
:1030500029BB316A431AE31838BF1C469368A34260
:1030600002D9081900F02CFB73699A6894420CD8B5
:103070005A68AC602B606A6015609A685D60121BCC
:103080009A604FF0FF33F36170BD1B68A41AECE740
:103090000C37002038B51B4C636998420DD0D0E93D
:1030A000003213605A6000228168C2609A680A4444
:1030B0009A604FF0FF33E36138BD2246036842F85F
:1030C000143F002193425A60C16003D1BDE83840EB
:1030D00000F0F0BA9A688168256A0A449A6000F0A4
:1030E000F3FA63699A68411B8A42E5D9AB181D1A45
:1030F000092D206A98BF01F10A02BDE8384010444A
:1031000000F0DEBA0C3700202DE9F041184C002702
:1031100004F11406656900F0D7FA236AAA68C11A97
:103120008A4215D813442362D5E9003213605A60ED
:103130006369D5F80C80EF60B34201D100F0BAFAB0
:1031400087F311882869C047202383F31188E1E7BA
:103150006169B14209D013441B1ABDE8F0410A2B42
:103160002CBFC0180A3000F0ABBABDE8F08100BF38
:103170000C37002000207047FEE700007047000079
:103180004FF0FF3070470000BFF34F8F024AD36803
:10319000DB03FCD4704700BF003C024008B5094B7C
:1031A0001B7873B9FFF7F0FF074B1A69002ABFBFFE
:1031B000064A5A6002F188325A601A6822F4806224
:1031C0001A6008BDC8380020003C02402301674552
:1031D00008B50B4B1B7893B9FFF7D6FF094B1A695B
:1031E00042F000421A611A6842F480521A601A686A
:1031F00022F480521A601A6842F480621A6008BD94
:10320000C8380020003C02400728F0B516D80C4C06
:103210000C4923787BB90C4D0E4608234FF0006211
:1032200055F8047B46F8042B013B13F0FF033A44A6
:10323000F6D10123237051F82000F0BD0020FCE7F7
:10324000EC380020CC380020583D0008014B53F8E2
:1032500020007047583D000808207047072810B527
:10326000044601D9002010BDFFF7CEFF064B53F8EE
:1032700024301844C21A0BB90120F4E71268013255
:10328000F0D1043BF6E700BF583D0008072810B511
:10329000044621D8FFF778FFFFF780FF0F4AF3239A
:1032A000D360C300DBB243F4007343F00203136145
:1032B000136943F480331361FFF766FFFFF7A4FF40
:1032C000074B53F8241000F02BF9FFF781FF20463D
:1032D000BDE81040FFF7C2BF002010BD003C024017
:1032E000583D0008F8B512F00103144642D1851884
:1032F0002E4A954257D82E4B1B6813F0010352D02B
:103300002C4DFFF74BFFF323EB60FFF73DFF40F23F
:103310000127032C15D824F001046618254C401A07
:1033200040F20117B142236900EB010524D123F0DB
:1033300001032361FFF74CFF0120F8BD043C04307A
:10334000E7E78307E7D12B6923F440732B612B69EF
:103350003B432B6151F8046B0660BFF34F8FFFF7BF
:1033600013FF03689E42E9D02B6923F001032B6110
:10337000FFF72EFF0020E0E723F440732361236969
:103380003B4323610B882B80BFF34F8FFFF7FCFE7D
:103390002D8831F8023BADB2AB42C3D0236923F094
:1033A00001032361E4E71846C7E700BFFFFF0708F2
:1033B00000380240003C0240084908B50B7828B1AB
:1033C0001BB9FFF7EBFE01230B7008BD002BFCD0EF
:1033D000BDE808400870FFF7FBBE00BFC8380020FA
:1033E00070B582B0FFF77EFD0E4E054600F06CF919
:1033F0003268904237BF0C4A0B49516814682EBF9F
:10340000D1E90041013151600419034641F1000145
:10341000284601913360FFF76FFD0199204602B005
:1034200070BD00BFF0380020F838002070B582B0C1
:10343000FFF758FD104E054600F046F932689042FD
:1034400037BF0E4A0D49516814682EBFD1E90041BB
:1034500001315160041941F10001034628460191F0
:103460003360FFF749FD01994FF47A72002320463B
:10347000FCF7B6FE02B070BDF0380020F83800202E
:1034800010B50244064BD2B2904200D110BD441C8C
:1034900000B253F8200041F8040BE0B2F4E700BF9B
:1034A000502800400F4B30B51C6F240407D41C6F0C
:1034B00044F400741C671C6F44F400441C670A4CFD
:1034C000236843F4807323600244084BD2B29042D5
:1034D00000D130BD441C00B251F8045B43F82050C9
:1034E000E0B2F4E70038024000700040502800408D
:1034F00007B5012201A90020FFF7C2FF019803B020
:103500005DF804FB13B50446FFF7F2FFA04205D0B7
:10351000012201A900200194FFF7C4FF02B010BDF1
:1035200070470000074B45F255521A6002225A605C
:1035300040F6FF729A604CF6CC421A60024B0122B0
:103540001A7070470030004001390020034B1B788F
:103550001BB1034B4AF6AA221A60704701390020BA
:1035600000300040044BD3F874389B0042BF034B3B
:1035700001221A70704700BF00300240003900205D
:10358000024B4FF08072C3F874287047003002403D
:10359000014B1878704700BF00390020EFF3098312
:1035A00005494A6B22F001024A63683383F30988B4
:1035B000002383F31188704700EF00E0202080F3A0
:1035C000118862B60C4B0D4AD96821F4E0610904F8
:1035D000090C0A43DA60D3F8FC20094942F08072F2
:1035E000C3F8FC200A6842F001020A601022DA7770
:1035F00083F82200704700BF00ED00E00003FA05E9
:10360000001000E010B5202383F311880E4B5B6897
:1036100013F4006314D0F1EE103AEFF30984683C20
:103620004FF08073E361094BDB6B236684F30988F9
:10363000FFF708FC10B1064BA36110BD054BFBE77B
:1036400083F31188F9E700BF00ED00E000EF00E030
:103650003B0600083E06000870470000FEE7000039
:103660000A4B0B480B4A90420BD30B4BDA1C121A35
:10367000C11E22F003028B4238BF00220021FDF759
:10368000AFBE53F8041B40F8041BECE77C3E000877
:1036900084390020843900208439002070470000DC
:1036A00000F080B84FF08043002258631A61022274
:1036B000DA6070474FF080430022DA607047000004
:1036C0004FF08043586370474FF08043586A70470B
:1036D0004B6843608B688360CB68C3600B69436150
:1036E0004B6903628B6943620B680360704700009B
:1036F00008B5234B23481A6942F0FF021A611A6980
:1037000022F0FF021A611A691A6B42F0FF021A6373
:103710001A6D42F0FF021A651B4A1B6D1146FFF736
:10372000D7FF02F11C0100F58060FFF7D1FF02F125
:10373000380100F58060FFF7CBFF02F1540100F57E
:103740008060FFF7C5FF02F1700100F58060FFF7B0
:10375000BFFF02F18C0100F58060FFF7B9FF02F1B5
:10376000A80100F58060FFF7B3FF02F1C40100F586
:103770008060FFF7ADFFBDE8084000F097B800BFDC
:103780000038024000000240783D000808B500F013
:1037900009FAFFF785FBBDE80840FFF7E3BE00002C
:1037A00070470000104B1A6C42F001021A641A6E46
:1037B00042F001021A660D4A1B6E936843F0010342
:1037C00093604FF080432F229A624FF0FF32DA620B
:1037D00000229A615A63DA605A6001225A61082114
:1037E0001A601C20FFF74EB800380240002004E0A9
:1037F0004FF0804208B51169D3680B40D9B2C94374
:103800009B07116107D5202383F31188FFF768FB1D
:10381000002383F3118808BD08B5FFF7E9FFBDE871
:103820000840FFF7EFBE00001E4B1A6962F0FF026E
:103830001A611A69D2B21A614FF0FF301A695A69D7
:10384000586100215A6959615A691A6A62F08052B6
:103850001A621A6A02F080521A621A6A5A6A586226
:103860005A6A59625A6A1A6C42F080521A641A6E85
:1038700042F080521A661A6E0B4A106840F480704B
:103880001060186F00F44070B0F5007F1EBF4FF459
:10389000803018671967536823F40073536000F091
:1038A00061B900BF0038024000700040354B364A15
:1038B0001A64364A4FF4404111601A6842F001021E
:1038C0001A601A689107FCD59A6822F003029A6080
:1038D0002C4B9A6812F00C02FBD1196801F0F90127
:1038E00019609A601A6842F480321A601A6892036A
:1038F000FCD55A6F42F001025A67224B5A6F90076B
:10390000FCD5234A5A601A6842F080721A601F4A36
:1039100053685904FCD51B4B1A689201FCD51D4A0B
:103920009A600322C3F88C200022C3F894201A4B1B
:103930001A681A4B9A421A4B21D11A4A11681A4A2C
:1039400091421CD140F203121A60154A136803F029
:103950000F03032BFAD10B4B9A6842F002029A60D4
:103960009A6802F00C02082AFAD15A6C42F480429A
:103970005A645A6E42F480425A665B6E704740F257
:103980000372E1E7003802400004001000700040BC
:103990001060410800948838002004E01164002081
:1039A000003C024000ED00E041C20F41084A08B56A
:1039B000516913680B4003F00103536123B1054AB9
:1039C00013680BB150689847BDE80840FFF71ABE6E
:1039D000003C014004390020084A08B551691368C9
:1039E0000B4003F00203536123B1054A93680BB106
:1039F000D0689847BDE80840FFF704BE003C01408E
:103A000004390020084A08B5516913680B4003F0D7
:103A10000403536123B1054A13690BB150699847F8
:103A2000BDE80840FFF7EEBD003C0140043900202E
:103A3000084A08B5516913680B4003F00803536145
:103A400023B1054A93690BB1D0699847BDE8084096
:103A5000FFF7D8BD003C014004390020084A08B5F2
:103A6000516913680B4003F01003536123B1054AF9
:103A7000136A0BB1506A9847BDE80840FFF7C2BD12
:103A8000003C014004390020174B10B55A691C68EE
:103A9000144004F478725A61A30604D5134A936A59
:103AA0000BB1D06A9847600604D5104A136B0BB16E
:103AB000506B9847210604D50C4A936B0BB1D06B21
:103AC0009847E20504D5094A136C0BB1506C98472E
:103AD000A30504D5054A936C0BB1D06C9847BDE89B
:103AE0001040FFF78FBD00BF003C014004390020AB
:103AF0001A4B10B55A691C68144004F47C425A6190
:103B0000620504D5164A136D0BB1506D9847230515
:103B100004D5134A936D0BB1D06D9847E00404D5DA
:103B20000F4A136E0BB1506E9847A10404D50C4A8E
:103B3000936E0BB1D06E9847620404D5084A136F98
:103B40000BB1506F9847230404D5054A936F0BB10E
:103B5000D06F9847BDE81040FFF754BD003C0140CE
:103B600004390020062108B50846FEF78BFE062121
:103B70000720FEF787FE06210820FEF783FE0621B8
:103B80000920FEF77FFE06210A20FEF77BFE0621B4
:103B90001720FEF777FEBDE8084006212820FEF733
:103BA00071BE000008B5FFF73FFE00F00BF8FEF70E
:103BB0007FFEFFF77FF8FFF7F3FDBDE80840FFF752
:103BC0006FBD00000023054A19460133102BC2E9DE
:103BD000001102F10802F8D1704700BF043900203B
:103BE00010B501390244904201D1002005E003786C
:103BF00011F8014FA34201D0181B10BD0130F2E7AC
:103C00002DE9F041A3B1C91A17780144044603F124
:103C1000FF3C8C42204601D9002009E00578BD42D6
:103C200004F10104F5D10CEB0405D618A54201D12D
:103C3000BDE8F08115F8018D16F801EDF045F5D0DD
:103C4000E7E70000034611F8012B03F8012B002AD7
:103C5000F9D170476F72672E6172647570696C6F0D
:103C6000742E6269726463616E6479004E6F2061C4
:103C70007070207369670A00426164206677206C67
:103C8000656E6774682025750A0042616420626F62
:103C90006172645F69642025752073686F756C6458
:103CA0002062652025750A004261642066772064E1
:103CB000657363726970746F72206C656E67746887
:103CC0002025750A004261642061707020435243D0
:103CD000203078253038783A3078253038782030E0
:103CE00078253038783A3078253038780A00476FB0
:103CF0006F64206669726D776172650A0040A2E4A4
:103D0000F164689106000000000000007D2C0008AE
:103D1000692C0008A52C0008912C00089D2C000897
:103D2000892C0008752C0008612C0008B12C0008B3
:103D30006D61696E0000000069646C650000000040
:103D4000383D000850370020C8380020010000002E
:103D50009D2E000800000000004000000040000010
:103D600000400000004000000000010000000200D0
:103D700000000200000002000004802A0000000091
:103D8000AAAAAAAA00004001DFFF0000000000006C
:103D90000080080010000A00000000009AAAAAAAE9
:103DA00000000000FBFF0000000000008800000091
:103DB0000000000000000000AAAAAAAA000000005B
:103DC000FFFF0000000000000000000000000000F5
:103DD00000000000AAAAAAAA00000000FFFF00003D
:103DE00000000000000000000000000000000000D3
:103DF000AAAAAAAA00000000FFFF0000000000001D
:103E0000000000000000000000000000AAAAAAAA0A
:103E100000000000FFFF00000000000000000000A4
:103E20000000000000000000AAAAAAAA00000000EA
:103E3000FFFF000000000000000000000000000084
:103E4000000000000A000000000000000300000065
:103E50000000000000000000B8C3FF7F0100000068
:103E600014040000000000000000070064000000CF
:0C3E700000000000FE2A0100D204000047
:00000001FF
